:100000000C9434000C943E000C943E000C943E0082
:100010000C943E000C943E000C943E000C943E0068
:100020000C943E000C943E000C943E000C943E0058
:100030000C943E000C943E000C943E000C943E0048
:100040000C943E000C943E000C943E000C943E0038
:100050000C943E000C943E000C943E000C943E0028
:100060000C943E000C943E0011241FBECFEFD8E04C
:10007000DEBFCDBF0E94A5000C94FC000C940000D4
:10008000F894219A81E880938000E1E8F0E08DE027
:1000900080838FEF90E0909389008093880084B1F3
:1000A000866084B98081816080837894089580E837
:1000B00090E09093890080938800089588E090E014
:1000C000909389008093880008958FEF90E090933B
:1000D0008900809388000895579A1BB808955F9A05
:1000E00008955F9808959B01AC0184E0220F331FAF
:1000F000441F551F8A95D1F760E074E284EF90E0C9
:100100000E94DA00215031093093C5002093C400C9
:1001100088E18093C10086E08093C200E0ECF0E0CB
:1001200080818D7F808308959091C00095FFFCCFE2
:100130008093C60008958091C00087FFFCCF809116
:10014000C600089581E00C9494000E946C0060E861
:1001500075E280E090E00E9473000E94400000E899
:1001600010E088E0E82EF12CCFEFD0E00E949B0059
:100170008031C9F048F4843089F08830B9F7F092C2
:100180008900E092880013C0813229F0823271F731
:100190000E9471000CC00E946F0009C0109389007A
:1001A0000093880004C0D0938900C09388000E9407
:1001B000A200DCCFA1E21A2EAA1BBB1BFD010DC0C1
:1001C000AA1FBB1FEE1FFF1FA217B307E407F50707
:1001D00020F0A21BB30BE40BF50B661F771F881FE3
:1001E000991F1A9469F760957095809590959B0179
:0C01F000AC01BD01CF010895F894FFCFD1
:00000001FF
